:030000000219FDE5
:03000B000200AA46
:03002B0002016669
:03005B000202F9A5
:030073000202DFA7
:1000800002030406080C10182030406080040608A3
:100090000C10182030406080A0C000070F1F3F0DDB
:1000A0000D04050D050305030302C2AFC0D0C0E077
:1000B000206217E5256002E473E525F4F58A758B67
:1000C00000D262D0E0D0D0D2AF3285268AC262E5BB
:1000D00026F46036306803207210758B00D0E0D0B3
:1000E000D0C290C291C292D2AF32C290C291C2929B
:1000F000206E0D20660A7401D5E0FDE57EF4529075
:10010000758B00D0E0D0D0D2AF32758A00C28DD2CC
:1001100062210001B9306805206602D29001B93031
:100120006805206602D29101B9306805206602D2C6
:100130009201B9D29330680A2066077405D5E0FDB4
:10014000D29001B9D29430680A2066077405D5E0D0
:10015000FDD29101B9D29530680A2066077405D5A1
:10016000E0FDD29201B9C2AFC2AD53E6EFC0D0C03C
:10017000E0D2D3D2AFC2CEE52A6007207449152A57
:1001800021C77800790020742EE580307E01F4309C
:10019000E60278FF53DACF207E0343DA20307E0375
:1001A00043DA10C2D8C271E580307E01F430E60235
:1001B00079FFC3E89970CB306103752A1820740366
:1001C000752A18885FD27020740DE52B6004152BFA
:1001D00021D743DA01C2D82070024135A85F2061DF
:1001E00002C2702074367982B70431C3E894F040BB
:1001F0000374F0F8E8C4540F28F87984B703024177
:100200001CC313C3138721200802C313200A06C38B
:10021000C898F8411C28F8500374FFF88822E52D8F
:1002200054066011E533C313C31324062522F522B7
:1002300050037522FF7882B60459852224A824C36E
:10024000E52495644002A864C3E895664002A86668
:100250008825E56970024186C3E8AA699A5003E8D7
:10026000FAE4F9EAC333FBE56BF45B29400D256A38
:10027000F8E56A6002156A400B41860AC3E56A9A8E
:100280005002056A78FF8826C26EC3E52694F840BE
:1002900002D26EC3E52594404002D26420CF0AD03A
:1002A000E0D0D043E610D2AD32C2CF053A7801E5B6
:1002B0002A6005307402152AC3E55F940140057574
:1002C000620041D5756300756C00E5622401F5623A
:1002D00050037562FFD0E0D0D043E610D2AD32C2F9
:1002E000AFC0D053E67FC2607591008556948557A4
:1002F00095759104D0D0D2AF32C2AF53E6EFC2AD04
:10030000C0D0C0E0C0F0D2D3D2AFA8FBA9FCC2D805
:10031000307102616053DACF207E0343DA10307E01
:100320000343DA20D271E580307E01F420E60261D9
:100330003788278928A18D53DACF207E0343DA201E
:10034000307E0343DA10C2D8C271307402A17978CA
:1003500000E580307E01F430E602A179885FA1617A
:1003600053DACF207E0343DA20307E0343DA10C213
:1003700071206102813953DACF207E0343DA1030D5
:100380007E0343DA20C2D8D271885A895BC3E895CC
:1003900058F8E99559F97B007E087A00C3E8948CF7
:1003A000E994005005755E00812B882178A2E6A8AB
:1003B000216055C3E894C8E994005008E4D2E4FBF6
:1003C0007A0A8106C3E89468E994015008E4D2E30C
:1003D000FB7A0F8106C3E894D0E994025008E4D276
:1003E000E2FB7A1E8106C3E894A0E994055008E474
:1003F000D2E1FB7A3C8106C3E89498E9940850085E
:10040000E4D2E0FB7A787E00C3E8955CFCE9955D78
:10041000FD30E70AECF42401FCEDF43400FD755ED8
:1004200000C3EC9AED9E5003755E01885C895D8582
:100430005A58855B597802A161C3E89527F8E99578
:1004400028F9307C02A145307B02A145307A02A117
:100450003E207502815CE9FDE8FC817BE9C313F96C
:10046000E813F8307902A13EE9C313F9E813F83034
:0F0470007802A13EE9C313FDE813FC20612CC301
:10047F00EC941CED940240028192ED701EC3EC943B
:10048F00C850180529E52970021529C3E529940AD2
:10049F005002A179755F00D270A179E5296002152C
:1004AF00297888E6F97400207F087896B9030278D6
:1004BF009EE624FAFEE43400FFC3EC9EFCED9FFDA4
:1004CF009208B90310A2085007207609D27681E46A
:1004DF00307602C276A2085016B9030DECF424014F
:1004EF00FCEDF43400FD0204FE78007900A145B95B
:1004FF000315EC33FCED33FDC3EC940AFCED9400D3
:10050F00FD50047C007D00C3EC94FFED9400400689
:10051F0078FF7900A145EC8575F0A4C5F0A2F733FB
:10052F00F87900400302056178FF7900020561E95F
:10053F00C313F9E813F8307C0EE9600278FFC3E8C3
:10054F001338F8E43400F9C3E894FFE9940040024B
:10055F0078FF885FD270206102A179741FF4552F44
:10056F004BF52FC274EB7002D274752A18307403D6
:10057F00752A0A306102A18D20740353DAFE2074AC
:10058F0003752B06D0F0D0E0D0D0D2AD43E61032B9
:10059F0079010205BD79030205BD790A0205BD790E
:1005AF001E0205BD79640205BD79C80205BD781725
:1005BF00E4D5E0FDD8FAD9F6227A147B780205E467
:1005CF007A107B8C0205E47A0D7BB40205E47A0B7A
:1005DF007BC80205E47902B27DE4D294D5E0FDD266
:1005EF0091D5E0FDC291D5E0FDC294D5E0FDD2904A
:1005FF00E576D5E0FDC2907496D5E0FDD9D9EAF83D
:10060F00D5E0FDD8FBDBCED29422C37C007D0075F4
:10061F00F00005F0EA33FAEB33FB50F6EB13FBEA8D
:10062F0013FAC3E9FFE8FEE89AF8E99BF95004EFE3
:10063F00F9EEF8B3EC33FCED33FDD5F0DFEDF9EC6B
:10064F00F822E889F08A20D2D4F8A9F07B0030F79D
:10065F000B7BFFF42401F8E9F43400F9E88520F06E
:10066F00A4ADF0F8E98520F0A4AFF0FEED2EF974FB
:10067F00003FFA7C04C3EA13FAE913F9E813F8DC34
:10068F00F48BF030F70AE8F42401F8E9F43400F9B8
:10069F00E889F0C2D4F8A9F0227882B604030207E1
:1006AF0003C3E55F940140030206CD852224E4F5E0
:1006BF0045F546F547F548F549C26D0207037882BF
:1006CF00E6FCD26DE522F523783879C7AA40AB4115
:1006DF00C3EB13FBEA13FAEC146013C3EB13FBEA3F
:1006EF0013FAEC14146007C3EB13FBEA13FAD119D6
:1006FF008845894622C3E5459523F8E5469400F9D8
:10070F00500CC3E89480E994FF4016020734C3E805
:10071F00947FE994005003020734787F7900020731
:10072F0034788079FF884A894B22E54A2547F8E5D6
:10073F004B3548F9854B20E4300701F43549FA3041
:10074F00E709C3EA94F04015020772C3EA940F5009
:10075F000302077278FF79FF7A0F02077278007928
:10076F00007AF0C3E5249564500AC37401952450B0
:10077F000B020790E54B20E70E020790E54B30E7A1
:10078F0006884789488A492278A4E6FAC3E54A339E
:10079F00F8E54B33F9D151E930E70BC3E89480E921
:1007AF0094FF4013E1CAC3E8947FE994005002E13B
:1007BF00CA787F7900E1CA788079FFE820E715C30E
:1007CF00E52398F84009C3E8940140030207F17844
:1007DF00010207F1E8F424012523F840030207F191
:1007EF0078FF884C2278A5E6FAA848A949D151E9A3
:1007FF0030E70CC3E89401E994FF4016020825C3C3
:10080F00E894FFE99400500302082578FF7900026D
:10081F000825780179FFE920E715C3E54C98F840E2
:10082F0009C3E89401400302084C780102084CE820
:10083F00F42401254CF8400302084C78FF88242249
:10084F0078FFC26420693D206A12D264C3E54194E7
:10085F000A4009C3E52594405002C26479A1E760BC
:0E086F0023E541601F74FF8541F0848539F058
:10087D00306A0375F005A4F8C5F0600278FFC3E88F
:10088D0095675002A867886622C3E5409440E5410C
:10089D009401E56650031401A7046002F566220277
:1008AD0008AF2275E890227883E6FFE5E820ECF7A3
:1008BD00A8BDA9BE0573C3E57394084052757300B6
:1008CD00E9FA79A0E76044EA7007E574601B020855
:1008DD00EAC3E895746010E5745006600C140208C4
:1008ED00F60460F90208F6E574F574C394F6401B3E
:1008FD007564C0C394064013756480C39406400BA1
:10090D00756440C39406400375640075BB0E22E503
:10091D00642410500274FFF5647982B704022143F8
:10092D00C3A864E524985002A824C3E89566400244
:10093D00A86688258826E573B4070375BB10227455
:10094D003279A687F0A4C5F0A2F733F8C3E8956411
:10095D004002A86488228824882588268867227505
:10096D0040007541F022C2AF75C820A8CCA9CDAA10
:10097D003A30CF010A75C824D2AFAB3BAC3C883BB3
:10098D00893CC3E89BF8E99C206908F9306702416E
:10099D008821E5AD3D8A3DF9EA9DFA600478FF793D
:1009AD00FFAE3EAF3F8B3E8C3FC3EC9FFCC3E99C3B
:1009BD00F542A83BA93CC3E89EF8E99FF9C3E54180
:1009CD0013FBE54013FAE82AF540E93BF5415006E3
:1009DD007540FF7541FF412FAA40AB41AC40AD4181
:1009ED007E047F02C3EB940440021E1FC3EB9408E8
:1009FD0040021E1FC3ED13FDEC13FCDEF7C3EA9C92
:100A0D00FAEB9DFBEF6009C3E913F9E813F8DFF783
:100A1D00EA28FAEB39FB8A408B4150067BFF8B406D
:100A2D008B41C3EB94025002D2673069047F0341BE
:100A3D005A7892E6FFC3E537948240110FC3E5372C
:100A4D0094A040010FC3EF940640027F057E04E59C
:100A5D0041C4540FF9E541C454F0F8E540C4540FB6
:100A6D0028F8C3E89EFAE99400FB4009C3EA940212
:100A7D00EB940050047A02E4FB41D4AA40AB41EB65
:100A8D00C4FEEAC4540F4EFCC3EA9CFAEB9400FB7F
:100A9D00C3E813C313F8EA28FAEB3400FB8A408B42
:100AAD0041C3EB94024002C2677804EBC4FE7B00A5
:100ABD00EAC4540F4EFAC3EA98FA4005C3940250A3
:100ACD00027A027892E6FF30600241D48552568553
:100ADD005357D26043E680C3E49AF8E49BF930673C
:100AED0002616EE8FAE9FBD3E913FDE813FC8852C5
:100AFD008953C3EF94036038EF20E00DE82CF8E93B
:100B0D003DF9ECFAEDFB020B29E828F8E939F9C3B8
:100B1D00E82402F8E93400F97AFE7BFFC3EF940371
:100B2D00400E8A548B55884E894F8C508D5161A241
:100B3D00885489558A4E8B4F8C508D51306920C306
:100B4D00E53394034019E542A2E713F8E555F42483
:100B5D000138400B20E7087554FFF42401F5556169
:100B6D00A2E8FAD3E813FC8852C3EF94036020EF98
:100B7D0020E007E82CF8ECFA618EE8282402F87AD8
:100B8D00FEC3EF940340088A54884E8C5061A288AE
:100B9D00548A4E8C50E56BC3335002646BF56B3049
:100BAD00600261AC753402D26043E680E52D5406D7
:100BBD006026A840A941C3E913F9E813F8C2AF5361
:100BCD00E67F759100C3E498F594E499F5957591D8
:100BDD0004D26043E680D2AF22D265754400752001
:100BED0000306B03752040020C05D265754400750D
:100BFD002040306B03752000D2AF7801206722E5CD
:100C0D002D54066002C265C3E54194054013780278
:100C1D0094054008780394054002780630690278FF
:100C2D000A206019E544601530690AC3E533940361
:100C3D004003D53406D2AFD26C81D771B4D2AF0098
:100C4D0000C2AF206726E541C3FB940F40027B0F26
:100C5D00EB240530730123306A02742820620123CE
:0E0C6D00F93069027982E58BC39940B50544E0
:100C7B00E59BF45440B5200281C130690A08C3E8F2
:100C8B00940A400108812E2065028105C26553E656
:100C9B007F7591003067107594007595FE75910402
:100CAB00D26043E6808105AE40AF41C3E49EF5942C
:100CBB00E49FF59581A8C3E533940250028105307A
:100CCB0065028105D80281D5812EC26C53E67F75F2
:100CDB009100855494855595759104854E56854F95
:100CEB0057D26043E680D2AFE52D54066008206AE8
:100CFB00020533020D11306C0D206B0A20650715B0
:100D0B0081158102157C22780030640530650278EC
:100D1B0001E53775F007A4F9E5F028F5F0E9A2F045
:100D2B0013A2F113A2F213F537C39478500375375E
:100D3B0078C3E53795384008D266C290C291C2920B
:100D4B00306002A14B855056855157D26043E680E7
:100D5B0022207D11C2AF754302D294C293D2AF75DC
:100D6B009F11020F2BC2AF754302D294C295D2AF23
:100D7B00759F11020F2B307243207D20C2AF75433C
:100D8B0003900144757E10C292D295306204D291C9
:100D9B00A19FC294D2AF759F01020F2BC2AF7543B7
:100DAB0003900144757E10C290D293306204D291AD
:100DBB00A1BFC294D2AF759F21020F2B207D17C20A
:100DCB00AF75430390011FC292306202D291D2AF32
:100DDB00759F01020F2BC2AF75430390011FC29089
:100DEB00306202D291D2AF759F21020F2B207D1161
:100DFB00C2AF754304D293C295D2AF759F21020F38
:100E0B002BC2AF754304D295C293D2AF759F01022B
:100E1B000F2B307243207D20C2AF754305900133F9
:100E2B00757E08C291D294306204D290C13BC293BA
:100E3B00D2AF759F11020F2BC2AF754305900155B1
:100E4B00757E20C291D294306204D292C15BC2955E
:100E5B00D2AF759F11020F2B207D17C2AF754305C3
:100E6B00900115C291306202D290D2AF759F1102E0
:100E7B000F2BC2AF754305900129C2913062EBD2A3
:100E8B0092D2AF759F11020F2B207D11C2AF75430C
:100E9B0006D295C294D2AF759F01020F2BC2AF75CC
:100EAB004306D293C294D2AF759F21020F2B30729F
:100EBB0042207D20C2AF754301900155757E20C243
:100ECB0090D293306204D292C1D7C295D2AF759FA4
:100EDB0021020F2BC2AF754301900133757E08C2FF
:100EEB0092D295306204D290C1F7C293D2AF759F64
:100EFB0001E12B207D16C2AF754301900129C290F1
:100F0B00306202D292D2AF759F21E12BC2AF7543F3
:100F1B0001900115C292306202D290D2AF759F013F
:100F2B00C26622900113757E00C290C291C292D20A
:100F3B0093D294D295C262227880760908760908FA
:100F4B0076040876FF0876030876FF08760B08769A
:100F5B0003087601087601788C76010876FF08760F
:100F6B00FF0876FF0876FF0876FF0876030876FF02
:100F7B000876FF0876FF0876250876D008762808CD
:100F8B0076500876040876FF087602087600087615
:100F9B007A0876FF08760108760108760008760352
:100FAB00227887E6FFC272BF0302D2727888E6C34B
:100FBB0094036008C27DE630E102D27DC27E78895F
:100FCB00E630E102D27EC3EF94026008758E01D247
:100FDB0073020FE4758E00C273227880E6149000C2
:100FEB00809378A4F67881E6149000809378A5F628
:100FFB007886E61490008D9378A6F6789CE6753883
:10100B00FF75390CB402067538A075390AB403069E
:10101B0075388275390578A3E61490009A93F569B3
:10102B00120F2E22227896E6FA7897E6FB7888E65E
:10103B00B40305C3EB940EFB307F047A007BFFC334
:10104B00EB9AFCC3948250027C827575000575EC9B
:10105B008575F0A4C3E5F0947D40F222D27F113068
:0F106B001205AE7A007B007C101205A4E55F2A07
:10107A00FA74003BFBDCF37C04C3EB13FBEA13FAC0
:10108A00DCF7FEC27F113022E5EF20E6037520006F
:10109A000520903FFFE520146006901DFF146000B4
:1010AA009304600375EF1053D9BF7581C043FF8065
:1010BA0012059F75EF0043B203E5B3240420E70D40
:1010CA00F521E5E320E0068521B343E301120F2E63
:1010DA007580FF75A40075F1D075D4BF75907875C9
:1010EA00A53F75F2BF75D54075A60175E241E4F8D2
:1010FA00F6D8FD756B01120F431215BE78988676E5
:10110A00753001C2AF1205B81205C81205AE120534
:10111A00CF1205AE1205D61205AEC2AF78FA79FA29
:10112A00308607D9FBD8F7021C00120FAC120FE564
:10113A00112F113078988676120F2E75885075897E
:10114A001275C82475910475D84075A82275B8021D
:10115A0075E690759B80759D0075D10775BC5875AD
:10116A00BB0E75BA1175E88012059FD2AF1208AC92
:10117A0053DACF207E0343DA20307E0343DA10436A
:10118A00DA01C2D8C2711205B8D2617B037A0CE5C2
:10119A005E70077A0CDB030211241205AE2070037D
:1011AA00021124C270E55FC3940240E1E52F541F87
:1011BA00856160F561B560D5DAD5C26153DACF20B1
:1011CA007E0343DA20307E0343DA10C2D8C2717834
:1011DA00A2E67008D274E52F54E0F52FC27575297E
:1011EA00001205B3307409C3E529940A4002D27586
:1011FA001205A478023074027800C3E55F9840F0C3
:10120A00C2AF1205C81205C81205C8D2AF1205B876
:10121A00754D007888E6B4030241FB1205A4788C68
:10122A00E6C3940150030212FBE530C39401500354
:10123A000212FB207435C3E55F94FF50030212FBD0
:10124A00C2AF1205DDD2AF1205B3C3E55F940150F8
:10125A00EFC2AF1205C81205A91205C8D2AF12050E
:10126A00B3C3E55F94FF40E90217667F02D27F119C
:10127A00301205B3C2AFC27F1130AE5FC3E55F94CF
:10128A007FD2AF407612059FC2AF1205DDD2AFDF23
:10129A00DC1167C3EE94057897F61205B8121600AA
:1012AA001216E97F0AD27F11301205B3C2AFC27F8C
:1012BA001130AE5FC3E55F947FD2AF50E612059F4F
:1012CA00C2AF1205C81205A91205C8D2AFDFD611DE
:1012DA0067EE24057896F61205B81216001217184A
:1012EA001205B31130C3E55F94FF5002413D021766
:1012FA0066C3E55F954D4003855F4D1205B37801DE
:10130A007988E7B403027805C3E55F984002411D76
:10131A00C2AF1205DD1205DD1205DDD2AF1205B826
:10132A00753000E4F531F5320531E531F4703905EF
:10133A0032789AE67819146012783214600D787D42
:10134A0014600878FA146003753200C3E5329840D5
:10135A001715327531B478998676C2AF1205DDD287
:10136A00AF789886761205B31205A9E52A7005307A
:10137A007402212478012074027806C3E55F98403C
:10138A00A77888E6C3940360031205B3E52A7003BD
:10139A00021124C2AF120F2EE4F522F523F524F52B
:1013AA0025F526F56AD2AF7885E6C333F568E4F504
:1013BA0045F546F547F548F549F573F52CF52DF54C
:1013CA003775730875BB1012059F1208B0E5E8203F
:1013DA00ECFBA8BDA9BEE97001F888741208B475BF
:1013EA00730875BB107887E6FE7602120FAC788711
:1013FA00EEF6C2AF7564FF12094C85226485226538
:10140A00852266D2AF7522017524017525017526DC
:10141A000185636C756D017888E6B40307C27D3077
:10142A007602D27DD268D269753300120E94120EFA
:10143A00B912096C12097312096C12097312096C38
:10144A0002145AC2AF120FACD2AF75730075BB0E3D
:10145A00120BF71206A8120D12120D5C1209731262
:0E146A000BE6306D0312070420670312084FD3
:10147800306703120896120D12120D8112097312A9
:101488000BF7306D03120739120D12120DF81209FD
:1014980073120BE6306D03120797120D12120E1D10
:1014A800120973120BF7306D031207F4120D1212A2
:1014B8000E941209731208B0120BE6120D12120ED6
:1014C800B91208B4120973306935206B3285676424
:1014D80085676585636C756D0179187A0CC3E5338A
:1014E80099400FC269D26A8A358567648567660242
:1014F8001507C3E55F9401400302145A02158430AE
:101508006A1B206B18E535147004C26A814DF535E5
:10151800C3E55F9401400302145A0215847536002E
:10152800C3E56278FA985054307404E52A604D781F
:1015380088E6B40317207D05207607A1543076028B
:10154800A154206B07D26B856764819978F0306B62
:10155800058567647820C3E541985002815A306B4D
:101568001BC26BC27D307602D27DD26A7535128578
:101578006764815A0536E55F6002A187753600C247
:10158800AF120F2E7887E6FE7602120FAC7887EE40
:10159800F6E4F522F523F524F525F526F568C26865
:1015A800D2AF12059F120F2E307409C3E536940589
:1015B80040022124612D901A0D7820121642E52050
:1015C800B4550CA3121642E520B4AA030215E01282
:1015D8000F431216000215FF901A0378807B0A1237
:1015E8001642A308DBF9901A0F788C7B1812164262
:1015F800A308DBF9901A2722C2AF12168112165BD4
:10160800901A00740E121647A37404121647A37496
:1016180014121647901A0378807B0A121646A308FC
:10162800DBF9901A0F788C7B18121646A308DBF9A1
:10163800121694121672901A2722E493F622E643A1
:101648008F01538FFD75EF0275B7A575B7F1F0538C
:101658008FFE22438F02438F0175EF0275B7A57580
:10166800B7F1901A0DF0538FFC22901A0D7455D1D2
:1016780047901A0E74AAD147227A3079D0782090F0
:101688001A40D142E520F709A3DAF7227A3079D057
:10169800901A40E7D14709A3DAF922AB77A878BBBB
:1016A80001027980BB02027981BB03027982BB0403
:1016B800027984BB05027986BB06027992BB0702D0
:1016C8007987BB080279A3BB0902799CBB0A027916
:1016D80088BB0B027989E8F7227C051205B8DCFB88
:1016E80022C2AF1205C81205CF1205D61205DD12A7
:1016F80005A91205C81205CF1205D61205DD120577
:10170800A91205C81205CF1205D61205DDD2AF22DF
:10171800C2AF1205DD1205D61205CF1205C8120593
:10172800A91205DD1205D61205CF1205C81205A9A2
:101738001205DD1205D61205CF1205C8D2AF22AEAA
:1017480077AF78C2AF1205C81205C81205C81205CE
:10175800A9DEF21205DD1205A9DFF8D2AF22D1E920
:10176800D1E1D1E1757701757801757900F1477C90
:1017780005AD5F1205B8C3ED955F70F5C3E55F94DD
:1017880001400AC3E55F94FF40320217A2D1A3D1FA
:1017980000D1E9C2AF75EF10D1E1DCD50579C3E519
:1017A800799403500280C6D1E10578E5771490005A
:1017B8009F93F808C3E57898500280AED1E1D1E153
:1017C8000577C3E577940C5002809C120F43D10033
:0717D800C2AF75EF10D1E173
:0319FD0002109243
:101A00000E0414090904FF03FF0B03010155AA0189
:101A1000FFFFFFFFFF03FFFFFF25D0285004FF0259
:081A2000007AFF01010003FF41
:101A40002344503341232020202020202020202008
:101A500023424C48454C4923463333302320202031
:101A60002020202020202020202020202020202076
:101C0000C2AFC2D353D9BF7581C043B20343FF8073
:101C1000752438752503B1C975EF0275E24043F1AB
:101C20004053A4BF75D400D2867DFA780379E67C50
:101C300010752200752300901DD67B0675249875BB
:101C400025013086028142208608D8FBD9F9DCF7CD
:101C500081B4308608D8FBD9F9DCF781B4B189E4C6
:101C600093A3C39A6004DDC381B4DBDBB17B600264
:101C7000812B7B08E493FAA3B15CDBF87A30B15C8A
:101C8000752200752300B17BEAFCEBFDC3ED94FEE9
:101C9000400EB17B8A278B28ED30E0048A828B834B
:101CA000B17B7AC270D8C3ED94FE601350CEBD00F4
:101CB00025EC60097520007521FF0200008100A855
:101CC00027A9280809D804D90281D3B17FEA89AAB3
:101CD000F281C50D81A0C3ED94035049EDA2E092BD
:101CE000007AC5C3E5829400E583941C50902000DF
:101CF00010438F02438F0175B7A575B7F1F030001F
:101D00001FA827A9280809438F01538FFDD804D99C
:101D100002A12089AAE275B7A575B7F1F0A3A10DBC
:101D2000538FFC817C7AC1BD030CE493A3FAB140CC
:101D3000DCF8B138817C817EAA22AB23B15CEBFA5E
:101D4000EA6222752608C3E52313F523E52213F57D
:101D50002250066323A0632201D526EAB1C9B1C986
:101D600075260AEAF4200102D286300102C286B149
:101D7000C9C3134002C201D526EB22B17FEAFB2082
:101D80008602A17F308602A184752608AE24AF2585
:101D9000C3EF13FFEE13FEB1CDB1C9C3EA13308612
:101DA000024480FA30E703632201C3E52313F523DD
:101DB000E52213F52250066323A0632201D526D91C
:101DC000E52265236523F52222AE24AF250E0FDE22
:101DD000FEDFFCD20122424C48656C693437316326
:041DE000F3300601D5
:00000001FF
